:020000020000FC
:02000000E7C453
:10000C0000C00F930FB70F931F93EF93FF9361FFF4
:10001C00C3C06D7FE0E7F1E0019112B31F70012BBB
:10002C0002BB019108BB019105BB019112B31F707A
:10003C00012B02BB019108BB019105BB019112B3CD
:10004C001F70012B02BB019108BB019105BB0191F3
:10005C0012B31F70012B02BB019108BB019105BBB0
:10006C00019112B31F70012B02BB019108BB0191CE
:10007C0005BB0000019112B31F70012B02BB019153
:10008C0008BB019105BB04E00A95F1F700000000E4
:10009C00019112B31F70012B02BB019108BB01919E
:1000AC0005BB06E00A95F1F70000019112B31F7031
:1000BC00012B02BB019108BB019105BB07E00A951E
:1000CC00F1F700000000019112B31F70012B02BB6D
:1000DC00019108BB019105BB09E00A95F1F70000FD
:1000EC000000019112B31F70012B02BB019108BBE0
:1000FC00019105BB0BE00A95F1F7019112B31F704A
:10010C00012B02BB019108BB019105BB0CE00A95C8
:10011C00F1F700000000019112B31F70012B02BB1C
:10012C00019108BB019105BB0EE00A95F1F70000A7
:10013C000000019112B31F70012B02BB019108BB8F
:10014C00019105BB00E10A95F1F7019112B31F7003
:10015C00012B02BB019108BB019105BB01E10A9582
:10016C00F1F700000000019112B31F70012B02BBCC
:10017C00019108BB019105BB03E10A95F1F70191CF
:10018C0012B31F70012B02BB019108BB019105BB7F
:10019C006460E0EAF1E00AC0F201019112B31F7051
:1001AC00012B02BB019108BB019105BB019111917F
:1001BC001BBD0ABD2F01339601911191012B09F43E
:1001CC006360FF91EF911F910F910FBF0F911895E5
:1001DC00510055005A006000640069006E00720006
:1001EC0078007C00820086008B00900095009A00BD
:1001FC009F00A300A900AD00B200B700BC00C10075
:10020C00C600CB00CF00D500D900DE00E300E8002B
:10021C00ED00F200F600FC00000105010A010F01DF
:10022C00140119011E01220127012D013101360192
:10023C003B01400144014A014F01530158015D014A
:10024C00620167016C01710175017B017F01840101
:10025C0089018E01930198019C01A201A601AB01B9
:10026C00B001B501BA01BF01C401C801CE01D20170
:10027C00D701DC01E101E601EB01EF01F501F90128
:10028C00FF01030208020D02110217021C022002D8
:10029C0025022B022F02340238023E02430247028F
:1002AC004D02510256025B026002650269026F0246
:1002BC00730279027D02820287028C0291029502FE
:1002CC009B029F02A402AA02AE02B302B702BD02B5
:1002DC00C202C602CB02D102D502DA02DF02E3026D
:1002EC00E902ED02F302F702FC02010306030B0321
:1002FC00100314031A031E03230328032D033203D4
:10030C0037033C03400346034A034F03540359038A
:10031C005E03630367036D03710376037B03800342
:10032C0085038A038F03930398039E03A203A703F9
:10033C00AC03B103B503BB03C003C403C903CE03B1
:10034C00D303D803DD03E203E603EC03F003F50368
:10035C00FA03FF03040409040D04130417041C041A
:10036C00210426042B043004350439043F044304CF
:10037C0048044D04520457045C04600466046A0487
:10038C007004740479047E04820488048D0491043E
:10039C0096049C04A004A504A904AF04B404B804F6
:1003AC00BE04C204C704CC04D104D604DA04E004AD
:1003BC000FEF01BB07BB04BB02BB08BB05BBE0E6F0
:1003CC00F0E0002710E101931A95E9F7E0E7F0E07F
:1003DC000FEF019300271FEF01931A95E9F7626065
:1003EC0008950CD025D003E10BBD08E80ABD002709
:1003FC000FBD09E00EBD00E109BF0895A0E7B1E013
:10040C00C0E7D0E00027802E902EA02E2227099145
:10041C00002309F051D08D929D92AD9223952031FD
:10042C00B1F78092090290920A02A0920B020895F1
:10043C00C0E8D0E08090090290900A02A0900B02D4
:10044C0020E1A0EAB1E00CED11E0680105E612E054
:10045C0078010991002341F02FD0ED92FD928D92FD
:10046C009D92AD92EE24FF24F601459155916F01BA
:10047C008A010E0D1F1D30F4ED92FD928D929D920E
:10048C00AD928A01780123952F3F19F7F60145911A
:10049C0055918A010E0D1F1D30F4ED92FD928D9237
:1004AC009D92AD928A010D931D938D929D92AD926A
:1004BC0000270D930D930895E0E6F0E000E111E0C4
:1004CC003481321709F4912A3285321709F4A12AA2
:1004DC003191321709F4802A8894001F8894111FD7
:1004EC0016FFEECF0895ECE0F2E0002710E8019340
:1004FC001A95E9F70895008111810117C9F0C4819B
:10050C00D581278136814427C31BD40B328143818B
:10051C00DD2322F4020FC30FD41FFACFC483D5837B
:10052C00222312F0101701C0011708F4012F0083C9
:10053C000895E0E7F0E00027112701931395E9F700
:10054C000FEF0093B0000093F00000931001ECE06B
:10055C00F2E0A0E6B0E050E1CEDF00810D93C0E701
:10056C00D0E01127C00FD11F0FEF088338965A9592
:10057C0099F7089509811881011B11E010F4019578
:10058C001FEF0E831F83AA81BB811197B695A79588
:10059C00AC83BD830895ECE8F2E0002718E70193E3
:1005AC001A95E9F7CCE8D2E008EA17E0088319833A
:1005BC0000270A830B830C830D8308950AE0202EF9
:1005CC00CCE8D2E0E881F9810E2F0F2BA1F0AA81A3
:1005DC00BB810A2F0B2B61F405911591DF01F801FA
:1005EC00CF93DF930995DF91CF91E883F983EACF1D
:1005FC001197AA83BB832C962A9421F70895FD01A9
:10060C001C8105913196010FCCE0D2E018E0019FDE
:10061C00C00DD11D05913196088309830895FD0104
:10062C001C8105913196010FCCE0D2E018E0019FBE
:10063C00C00DD11D08810F3F09F003950883098374
:10064C000895FD011C8105913196010FCCE0D2E09B
:10065C0018E0019FC00DD11D0881002309F00A95F7
:10066C00088309830895FD011C8105913196010FC2
:10067C00CCE0D2E018E0019FC00DD11D0591319660
:10068C000983059115910A831B830E94C00208956A
:10069C00FD01A591B591AA83BB830895FD01A59198
:1006AC00B591FD01EE0FFF1F0895FD010D81033083
:1006BC0080F4102F13951D83000F11271296C00F75
:1006CC00D11FAE83BF83A591B591FD01EE0FFF1F26
:1006DC0001C032960895FD010D81002349F00A9561
:1006EC000D83000F1127C00FD11FEE81FF8102C0B7
:1006FC00EE27FF270895FD01A591B591AA0FBB1F09
:10070C00059131961AE0CCE8D2E028813981232B6F
:10071C0021F02C961A95C9F707C0A883B983112725
:10072C001A831B830C831D830895EE27FF270895DE
:10073C00FD01A591B5910C9115913196A591B591AD
:10074C0021E0112319F01A95220FFBCF022319F087
:10075C00FD01EE0FFF1F0895FD01A591B5910C91C0
:10076C0015913196A591B59121E0112319F01A95A7
:10077C00220FFBCF022319F4FD01EE0FFF1F08958A
:10078C00FD01A591B5910C9115913196A591B5915D
:10079C00011719F4FD01EE0FFF1F089581033004BA
:1007AC0000004E030A0081033E0401004E030A00C0
:1007BC008103580402004E030A00810372040300F3
:1007CC004E030A0081038C0404004E030A008103CB
:1007DC00A60405004E030A008103C00406004E0364
:1007EC000A008103DA040700050308002000050352
:1007FC000900400005030A00600005030B0080009F
:10080C0005030C00A00005030D00C00005030E003D
:10081C00E00005030F00FF004E0332000503080043
:10082C00010005030900020005030A00030005038B
:10083C000B00040005030C00050005030D00060069
:10084C0005030E00070005030F0008004E033200DD
:10085C005403FA0339030000FF000A004E030A0098
:10086C003903000000001E004E03820054033004C4
:10087C0039030000FF000A004E030A003903000090
:10088C0000001E004E036E0039030000FF000A003A
:10089C004E030A0039030000AA000A004E030A00A6
:1008AC0054033E0439030000FF000A004E030A0003
:1008BC003903000000001E004E035A0039030000EB
:1008CC00FF000A004E030A003903000000001E005E
:1008DC004E031E005403580439030000FF000A00A5
:1008EC004E030A003903000000001E004E034600B0
:1008FC0039030000FF000A004E030A003903000010
:10090C0000001E004E033200540372043903000031
:10091C00FF000A004E030A003903000000001E000D
:10092C004E03320039030000FF000A004E030A0098
:10093C003903000000001E004E03460054038C04D3
:10094C0039030000FF000A004E030A0039030000BF
:10095C0000001E004E031E0039030000FF000A00B9
:10096C004E030A003903000000001E004E035A001B
:10097C005403A60439030000FF000A004E030A00CA
:10098C0039030000AA000A004E030A0039030000D4
:10099C00FF000A004E030A003903000000001E008D
:1009AC004E036E005403C00439030000FF000A001C
:1009BC004E030A003903000000001E004E038200A3
:1009CC005403DA040FE50DBF04E00EBF66270E9446
:1009DC00DE010E9479020E94D1020E94F7017894F4
:1009EC0062FFFECF6B7F0E94040260FFFECF6E7F22
:0E09FC000E941E020E94E4020E949F02F1CFA0
:00000001FF
